:1000000000308A0004280000840183131F30830518
:10001000193083169900A63098009030831298000A
:1000200083161F149F141F159F1107309C00FF306B
:100030008312A00083161F109F141F159F151F13F6
:1000400083121F179F1383169F1383121F1494127A
:10005000A01220088316870083122016200883161A
:1000600087008312A01120088316870001308312B5
:1000700094000030831694000108C73908388100C5
:10008000831290010030F800920000308316920035
:1000900007309C00050864000230F700F70B4E287B
:1000A00051281C0883120D1383169D014030F8005F
:1000B00083121F08C73978049F0064000630F700D8
:1000C000F70B60281F151F1963281E08A100A1083F
:1000D00003197B282108273C031C7B2883168511E4
:1000E00083128511831685128312851283160511DA
:1000F000831205150A292108273C0318B028210876
:100100003B3C031CB028831685128312851283168C
:1001100005118312051564002030F700F70B8E28B7
:100120009128831605118312051164002030F70011
:10013000F70B98289B28831685118312851164007C
:100140002030F700F70BA228A5288316851183120B
:10015000851564002030F700F70BAC28AF280A297A
:1001600021083B3C0318C52821084F3C031CC52827
:1001700083168512831285128316051183120511C9
:1001800083168511831285150A2921084F3C03180F
:10019000FA282108633C031CFA28831605118312F0
:1001A0000511831685128312851664002030F7002E
:1001B000F70BD828DB28831685128312851264007A
:1001C0002030F700F70BE228E5288316851183120B
:1001D000851164002030F700F70BEC28EF28831618
:1001E00085118312851564002030F700F70BF6287F
:1001F000F9280A292108633C03180A2983160511E6
:1002000083120511831685118312851183168512B9
:080210008312851662286300C9
:02400E0039393E
:00000001FF
